:020000040800F2
:106000002D482C49384A01602C4941602C49816057
:106010002C49C1602C4901612C4941612C498161A5
:106020002C49C1612C4901622C4941622C49816291
:106030002C49C16200F180012C4BCA6143632C4B97
:1060400083632C4B03632C4BC3632C4B03642C4B9B
:1060500043642C4B83642C4BC3642C4B03652C4B47
:1060600043652C4BC3662C4B83652C4B03662C4B32
:10607000C3652C4B43662C4B83662C4B03672C4B20
:1060800043672C4B83672C4BC3672C4808602C4814
:1060900008612C4848602C4848612C48C1E902023C
:1060A0002B488861704710B500F06AFB00F01DFCBA
:1060B000002010BD8D7500085C0400205976000892
:1060C00041720008F17600089B910008597700089A
:1060D0007B7700089D7700082DA100089F720008BB
:1060E000FB7A000841A50008076400082162000847
:1060F000696500080D7D00089D7100087D6B000832
:106100004B920008537100084D640008FF640008BA
:10611000F58C0008EF710008CD6E0008C565000819
:10612000DB65000809A400081F6E0008E98F00085D
:10613000237D0008237400085F940008A5A00008D0
:10614000AD9300081DA1000845710008D5A0000806
:10615000CF910008202802D94FF0FF307047B64A8F
:10616000102802EB400204D932F8220D61F31F20FF
:1061700004E032F8020D00F47F4008431080002054
:106180007047AD4A00204FF6FF7122F81010401CF6
:10619000C0B20F28F9D97047F0B50C46A74908449A
:1061A000A1F1240710F8013C581DC6B20A2594FB42
:1061B000F5F005FB104094FBF5F4C0B2202B01D89C
:1061C000B34202D94FF0FF30F0BD395C18465B1C7A
:1061D000DBB2FFF7BFFF002CE9DC0020F0BD9749E0
:1061E000A0F141023E390144192A02D811F8410CAC
:1061F0007047A0F16102192A02D811F8610C7047AA
:10620000A0F13001092901D8C8B270472D2803D068
:106210002E2803D02320704721207047222070476A
:10622000F0B5864E00240D460346243E834F16E00B
:10623000FFF7D5FF315CF81810F8010CFFF78AFF63
:106240005B1CDBB2202B02D94FF0FF30F0BD052CD8
:1062500001D00B2C01D19B1CDBB2641CE4B2285D85
:106260000028E5D1F0BD70B5044673480D462030D6
:10627000FDF7DCFC2846FDF7FDFC7049C0B29A39F9
:10628000012388704D7900222DB12044401EC87032
:106290004A700B7103E0CC70401E48700A714A715D
:1062A0008A71CB710B7070BD2DE9F0470346FFF783
:1062B00068FFDFF888A1DFF88891AAF1240AA3B368
:1062C0004FF00008002524E000241AE05B4F5346FD
:1062D0001AF80510385DFFF73DFF3E19595D307C17
:1062E000FFF738FFC82003F0DDFE385DFF21FFF720
:1062F00031FF307CFF21FFF72DFF641CE4B20F2C2F
:1063000003D899F800000028E0D06D1CEDB21E2DD6
:1063100003D899F800100029D6D008F1010000F048
:10632000FF08B8F10F0FCDD927E0FFE7002556464B
:106330004FF4C8784F46002418E00023315D18461A
:10634000FFF708FF5B1CDBB21E2BF7D9404603F0BA
:10635000A9FE0023FF211846FFF7FCFE5B1CDBB201
:106360001E2BF7D9641CE4B21D2C02D83878002803
:10637000E3D06D1CEDB2282DDDD999F8000010B9DD
:10638000304901200860FFF7FCFE2C4901207D39CF
:10639000FFF746FFBDE8F0472849613909203FE78C
:1063A000254810B5182228492030FDF78EFC2349D6
:1063B00000209A390870BDE81040E2E6F0B51E4DA5
:1063C0001E4E00232035243E06F14407A6F1760434
:1063D00010E0102B03D9C3F11800285C00E0E85C42
:1063E000FFF7FDFE315C2078C01A385CFFF7B2FE83
:1063F0005B1CDBB220788342EBD9C0B2401C20701A
:10640000F0BD7047704710B50B4C0021203400F0F0
:106410000F02C1F105030009E254092A01D94132F2
:1064200000E03032491CC9B2E2540629EFD3002003
:10643000A0710148203010BD780900200A03002017
:1064400044080020480800204B0A002070B57C4D0D
:10645000420716D50C0901F00F01820702D5285D0D
:10646000484005E0C00705D0285DC1F10F01084094
:10647000285500E02955734E30887349C00724D150
:1064800020E0242902D94FF0FF3070BD4A1ED317F7
:1064900002EB9372C2F3870422F00302491E8A1AA8
:1064A00001219140C9B2C20702D0285D084305E02E
:1064B0008007285D01D5484000E08843285500F05A
:1064C0000F00D5E70888C00708D03088C007FCD186
:1064D0000888C007F9D1052003F0FCFD5B48C168BE
:1064E0002A5D01F46F41D243120741EA1261214350
:1064F000C16001213046FAF789FE002070BD2DE908
:10650000F05F00244F4EDFF838A14FF0030BDFF8A7
:106510004081F025DFF830914C4F1AE0CCB1042CCB
:106520001DD0002132883046D207FBD1B9F80020B7
:10653000D207F7D1FA6802F46F4222430A43FA60A5
:106540000121FAF763FE641CE4B2092CE6D3BDE82E
:10655000F09F9AF800102BEA01000101E2E798F899
:10656000000025EA0001DDE72DE9F05F0024344D4D
:10657000344E4FF0030A4FF0C00BA046DFF8C8902E
:10658000324F19E0C4B1F02105F80480328830465A
:10659000D207FBD1B9F80020D207F7D1FA6802F48C
:1065A0006F4222430A43FA600121FAF72FFE641C6E
:1065B000E4B2092CE6D3CAE729782AEA01004BEABB
:1065C0000011E3E71E49002001F10A020B5C13549D
:1065D000401CC0B20928F9D3704770B5184D00248B
:1065E0000A35285D40EA0410C1B20420FFF72EFFEF
:1065F000641CE4B2092CF4D370BD70B5154C4FF493
:1066000096704FF4FA76144D20600FE0FFF777FF95
:10661000304603F047FDFFF7A7FF287810B9304652
:1066200003F040FD2168491E216002D0287800282F
:10663000ECD02878002801D10120206070BD000036
:10664000B109002000040040000800400010014093
:1066500081050020480800204408002070B5F54D51
:106660000420F549287102200870F44800240470C1
:10667000F348047003F0D6F8F349F2480860F34990
:106680000860F3486C70EC70047070BD10B5E94C94
:10669000012060712178C0B2FFF75CFD6079401C79
:1066A000C0B260712028F5D9207810B14000207068
:1066B00010BDFF20FBE7FEB5E64801241D2607C8F4
:1066C0008DE8070000272546684603F09DFE01E09F
:1066D000112C06D02146641CE4B20120FFF7B6FE5F
:1066E00000E012243146761CF6B20020FFF7AEFE21
:1066F000642003F0D7FC242C00D10124242E00D1E7
:1067000001267F1CFFB20A2F09D129466D1CEDB26C
:10671000002000F033FA092D00D10125002700F0F8
:1067200094FB0028D4D000F0B5FB0028D0D19DF810
:10673000000003F005FFFFF724FDC7A10120FFF7CC
:106740006FFDC9A10D20FFF76BFD0020FEBDC04904
:1067500010B501200870C84964200860C749086066
:10676000C749C84802F09AFBC7A10120FFF758FDAE
:1067700003F0D9F9FCF713FBBDE81040FFF701BDAA
:1067800070B5C348016841F4E0210160C1494FF48C
:106790007A700860C049DC200870C0490F2008707A
:1067A000FCF759FBFCF7D3FBFCF7A0FBFAF7FEF96B
:1067B000FCF71BFDFCF734FBFCF732FCFCF75FFC3D
:1067C000FCF788FCFCF708FCFFF71AFCB44800252E
:1067D000C0F8B4510121C0F8B011FCF726FBFDF759
:1067E00024FD30B9FDF77BFB0120FDF7B8FCFDF778
:1067F0007CFBAC480570FFF7C4FC00F0FEF9FFF726
:10680000B3FE00F02CFBFCF7D8FD03F01AFD03F0FB
:1068100074FCFFF723FF0020FCF7AAFAFCF72FFC1B
:10682000FCF758FC8A480078401E102802D300204C
:10683000FFF78DFFFCF709FA0020FCF7A4FA9A4C49
:106840009A4E2168884201D1307880B398A1012006
:10685000FFF7E6FC98A10920FFF7E2FC02F061FFD8
:1068600035700020FCF78FFA20600020FCF760FAFA
:106870004FF4487003F02EFC0020FCF784FA2168E6
:10688000884212D08EA10120FFF7CAFC8EA10920F8
:10689000FFF7C6FC4FF4C87003F01CFCFCF78DFD3D
:1068A000642003F017FCFCF788FDFFF76AFCFFF794
:1068B0005BFE87A10120FFF7B3FC87490B20FFF7A0
:1068C000AFFC86A11120FFF7ABFC864801681B20B6
:1068D000FFF7A6FC4FF4FA7003F0FCFB8248006857
:1068E000804702F01AFB002070BD804F564EDFF843
:1068F0004891DFF8FCB1DFF8FCA14FF000084D4CE7
:106900002079012801D0022819D1E078032814D178
:1069100079487A4900680978007A88420DD0784928
:10692000FCF712FD77A17C48FDF780F974497A489D
:10693000FDF7BFF97848FDF7F6F803F09EFD434DEB
:106940003168286888424CD000F0A4FAA070E17841
:1069500089B1FF280FD000F089FA6949FCF7F4FCEF
:106960006EA16D48FDF762F965496B48FDF7A1F925
:106970006948FDF7D8F899F800000228A07809D0F6
:10698000FF281ED0C0B2152807D0052808D802F06D
:10699000AFFE12E00328F5D913E002F08AFD0CE007
:1069A00000F064FA624909688847002805DAE0784F
:1069B000012802D15FA0FDF7B6F88BF800808AF8B5
:1069C0000080387850B96548007803F083FB286868
:1069D0003168884202D0A07800F078FA87F8008009
:1069E000AEE799F80000012813D19BF800102D297B
:1069F0000BD38BF80080E078012802D958A0FDF76E
:106A000092F85D480068804703E09AF800108BF820
:106A100000109AF80000544648B1224D2878012809
:106A200005D1FCF7FDFF85F8008084F8008001F0B7
:106A3000EAFA64E7AE0300209705002085030020F2
:106A4000440800202B0A0020500500204C0500209F
:106A500024040020ACA50008202020206E69777552
:106A60006D7066200000000020202041524D7072A1
:106A70006F6A656300000000300400202C040020D1
:106A8000140700200D070020202067616D650000BD
:106A900024ED00E0F8030020C0030020CF03002015
:106AA000000022421E0000203C040020CB030020F6
:106AB00020726573657400006E7672616D2000004F
:106AC000206E7672616D000073686F742020000084
:106AD00020702D72657600004506002020672D721B
:106AE0006576000038070020400700207A05002066
:106AF0002D0800202C0800204C0800205006002003
:106B0000C50900204576656E7420747269676765F3
:106B100072202D20000000009B0A0020537769742A
:106B2000636820436C6F736564202D2000000000B3
:106B30003C070020537769746368206E6F7420707F
:106B4000726F6772616D6D656420666F7220746824
:106B500069732067616D653F213F00000C070020CD
:106B60005761746368646F672042616C6C20536581
:106B7000617263682E000000FC0500202DE9F041E1
:106B80008446082937D88D4A8D481388DB07FCD105
:106B90000388DB07F9D18B4C5FEACC724FF001051B
:106BA000E2680FD04DF6FF731A404A40E2600027BA
:106BB000854E032910D9BCF1020F0DD20121FAF73D
:106BC00025FB14E002F45F434A1E05FA02F2C2F10B
:106BD000FF021343E360EAE7C6F8B451C6F8B471A4
:106BE000282003F077FAE06840F0FF00E060C6F884
:106BF000B451C6F8B471BDE8F081724810B5C168EF
:106C000041F0FF01C160704C0120C4F8B40104F5EB
:106C1000DA7403F047FA0020206010BD2DE9FC5F14
:106C20006AA00026D0E90010CDE9001001254FF43C
:106C3000487ADFF8A0814FF47A7BDFF89C91A8E0D6
:106C400066A10720FFF7ECFA01210020FFF7FEFB09
:106C5000C82003F03FFA01210846FFF7F7FB02F0D6
:106C6000DBFE00287BD15446504603F033FA02F095
:106C7000D3FE0028F6D15AA10720FFF7D1FA02214E
:106C80000120FFF7E3FBC82003F024FA02210020D3
:106C9000FFF7DCFB02F0C0FE00287FD1204603F0A6
:106CA00019FA02F0B9FE002878D14E48007890B168
:106CB0004DA10720FFF7B4FA11210120FFF7C6FB11
:106CC00098F8000003F006FA11210020FFF7BEFB40
:106CD000584603F0FFF902F09FFE00285ED14348BA
:106CE0000078B0B199F80000092812D040A107201F
:106CF000FFF796FA12210120FFF7A8FB98F8000091
:106D000003F0E8F912210020FFF7A0FB584603F03A
:106D1000E1F902F081FE10BB36A10720FFF780FAEF
:106D2000002423E06F461DF804100820FFF734FA12
:106D3000395D0020FFF722FF16B14FF4FA6000E042
:106D4000584603F0C7F900F0B7F8032803D100F064
:106D5000A1F82EB100262EB16D1CEDB204E01DE0AD
:106D60000126F8E7641CE4B2072C04D800F0A4F86C
:106D700008B1142DD6D399F80000092803D11221A7
:106D80000020FFF763FB00F06AF86D1CEDB2142DD4
:106D900004D802F041FE00283FF452AF02F03CFE5E
:106DA00010B915490120086001210020FFF74EFBB2
:106DB00010A10720FFF734FABDE8FC9F0004004053
:106DC00000080040001001400000224204050102BA
:106DD00003060708C0030020240400204C310000F3
:106DE0004C3200007D0500204C3300007E05002061
:106DF0004C34000020200000480800200A21B0FB8D
:106E0000F1F201FB1202B0FBF1F1C24B012088400C
:106E10009A5C024201D0002070470120704730B5D3
:106E2000BC4CBD4B0C3C2246A16852684FF0FF356C
:106E3000994201D11F3B00E04B1C9A4201D12846E8
:106E400030BD08700020A36030BDB2480C38D0E9D6
:106E50000110814201D00120704700207047AE48E8
:106E6000AC491F380C3988604860704700F00F014A
:106E7000000900EB800001EB4000C0B270470A211E
:106E8000B0FBF1F201FB1202B0FBF1F002EB0010DB
:106E9000C0B270479F4A0C3AD2E90110814201D139
:106EA000FF2070479C4B0878994202D1A3F11F0143
:106EB00000E0491C5160704796490C39D1E9010145
:106EC000884201D1FF2070470078704730B5914C5F
:106ED000914A0C3CFF23616809E00D78854200D19E
:106EE0000B70914202D18C491F3900E0491CA56802
:106EF000A942F2D130BD70B5884C0546207840B12A
:106F0000874E3078012804D1FCF78AFD00203070CC
:106F10002070804C0C3CD4E90101884209D12846FC
:106F200003F0C0F8D4E90101884202D14FF0FF30EC
:106F300070BDBDE87040ADE770B500254FF4167622
:106F40003046FFF7D8FFC4B2032C06D02CB16D1C1D
:106F5000EDB23C2DF4D3002070BD4FF4C870FFF7A4
:106F6000CAFF40B1032802D0032C0AD005E0032C4D
:106F700007D024B101E0032C01D0032070BD022012
:106F800070BD012070BD2DE9F041624E00254FF427
:106F900096773846FFF7AFFF040002D5F078C007B8
:106FA00008D0032C07D034B16D1CC82DF1DB0020B4
:106FB000BDE8F08103244FF4C870FFF79CFF40B197
:106FC000032802D0032C0AD005E0032C07D024B1FB
:106FD00001E0032C01D00320EAE70220E8E70120CA
:106FE000E6E710B5FFF7A8FF4E49087010BD10B5D1
:106FF000FFF7C9FF4B49087010BD464A0A210C3AF9
:107000001078B0FBF1F301FB1301052901D0401CFE
:1070100002E04B2802D0401D107070470020FBE7B3
:107020002DE9F0413B4E00250C3EDFF8FC803F4F40
:1070300064E04FF44870FFF75EFF040008D0032CB3
:1070400001D055B921E00DB1002557E0012555E0EB
:107050000020386052E0FFF7D0FF3078FFF7CEFE17
:1070600010B930780028F6D131A11520FFF7D8F8F3
:10707000317829B11620FFF78FF8FFF7BEFF3DE00A
:10708000012131702AA116202DE0002C2EDDE0B266
:10709000FFF7ECFE01461620FFF77EF81420FFF7FD
:1070A0002AFFA0422AD103210020FFF767FD012417
:1070B00020A10120FFF7B4F841460920FFF7B0F8FE
:1070C000FA2003F007F8FFF75CF8642003F002F8F9
:1070D000641C042CECDDFFF7C2FE18490120FFF709
:1070E0009FF841460920FFF79BF807E010A1152003
:1070F000FFF796F800211620FFF74EF83868401E7B
:107100003860401C95D1BDE8F0410DA11520FFF776
:1071100087B80000540500204A0A00202C080020EF
:107120001E00002079050020BE0200204808002033
:1071300020000000636C65616E2000008D0200205D
:107140002020000010B5FFF759FE002800D00120D4
:1071500010BD10B5FA4C60790A280AD3142801D35F
:10716000A07800E0607884F82200C1B20120FFF727
:107170006DF960790A21B0FBF1F201FB1200E064C5
:1071800000280AD021780844401EC1B284F8221099
:10719000BDE810400120FFF759B910BD10B5E84C0B
:1071A0006079142806D01D2804D00A2804D013289A
:1071B00002D007E0A17812E0617884F82210002064
:1071C000FFF744F960790A21B0FBF1F201FB1200EC
:1071D000E06400280AD021780844401EC1B284F837
:1071E0002210BDE810400020FFF730B910BD10B5E7
:1071F000D34C607994F82310884207D2FFF7CEFF72
:107200006079401C6071BDE81040A2E710BDCD4A16
:10721000CD4811780078814201D300280FD1491C54
:10722000C9B2117018B90F2901D90F201070C748C1
:107230000078002803D011781020FEF7ADBF70470A
:1072400010B504210020FFF799FCC148007868B10F
:10725000C0480068FDF749F80022BF4BFDF75CF815
:10726000FDF714F8BDE8104000F0DBB8BB48B54AA4
:107270000168491C0160B44910780978884201D33B
:1072800000290BD1401CC1B2B04811700078002811
:1072900004D0BDE810401020FEF77EBF10BD10B531
:1072A000AF48A74C007818B1217B206C884208D0E9
:1072B000AC48007810B1FFF7C3FF0AE000F066F9B0
:1072C00007E0A448006800F0ACF804210020FFF7B4
:1072D00055FC207B206410BD0246A34801680029AC
:1072E0000FDD8A420BDDA1480068884209DD824239
:1072F00006DD9F490968814203DD8A4201DA0846BA
:1073000070470020704710B59A4A8D4C1168607C18
:10731000491C012810D0022819D0032822D0E36E7E
:10732000002B2ADDA06E984227DD1160FFF7D4FF05
:10733000E066BDE81040B2E7636D002B1DDD206DF7
:1073400098421ADD1160FFF7C7FF6065F1E7E36D52
:10735000002B12DDA06D98420FDD1160FFF7BCFF1E
:10736000E065E6E7636E002B07DD206E984204DDE2
:107370001160FFF7B1FF6066DBE710BD704B10B521
:1073800018465A7C816F007A012A08D0022A0CD054
:10739000032A10D09A6E1144996690B114E01A6DC8
:1073A0001144196580B906200CE09A6D1144996565
:1073B00050B90E2006E01A6E1144196620B9162045
:1073C00000E01E20FEF7E8FEBDE810409BE75C48A9
:1073D0008030406C004710B5594CE07A00281FD12E
:1073E0000120E072A07B18B904210020FFF72EF8DD
:1073F00061480078002813D094F8330010B194F855
:10740000340002E094F8341021B118B94C488030AF
:10741000406C804759480078BDE8104003F090B8B0
:1074200010BD2DE9F0410446FFF7D5FF444DA87A81
:10743000002870D1012085F8370005F18000806BAD
:1074400080474F484FF47A764E4F0068E863B44265
:1074500033DB42F22830844216DC94FBF6F006FB64
:107460001040E8BB94FBF6F4387818B103210020F3
:10747000FFF784FBAE67FFF781FF641E002C4ADD37
:10748000E86B02F027FEEFE742F2107694FBF6F08D
:1074900006FB104020BB94FBF6F4387818B10521A8
:1074A0000320FFF76BFBAE67FFF768FF641E002C3D
:1074B0006ADDE86B02F00EFEEFE7642C1DDBB4F52D
:1074C000617F61DC642094FBF0F100FB114139B96C
:1074D00094FBF0F46426387828B10221002000E003
:1074E00015E0FFF74BFBAE67FFF748FF641E002C6B
:1074F0004ADDE86B02F0EEFDEDE70A2C07DB5A2CC3
:1075000042DC0A2094FBF0F100FB114121B1AC6791
:10751000BDE8F04132E737E094FBF0F40A26387812
:1075200018B101210020FFF729FBAE67FFF726FF06
:10753000641E002C28DDE86B02F0CCFDEFE70000B4
:1075400060050020D2030020D0030020C7030020E4
:10755000D5030020180400200000F83FF0030020AD
:10756000C1030020C2030020FC03002010040020FF
:107570001C04002008040020CE030020D4060020B4
:1075800030040020CD030020BDE8F08110B5FE4896
:10759000FE4C0078A17B884212D9FD48007820B1CA
:1075A000FC480068BDE810403BE704210120FEF7DD
:1075B0004DFFA07B401CA073F7480168491C016087
:1075C00010BD30B5F149F5488031F04C0A690068CA
:1075D000217CF34B50B1884208D91D68411A694398
:1075E000B1FBF0F1B2FBF0F2114401E092FBF1F1DA
:1075F0001960EC490A78002A2DD0EB490A2809685D
:1076000002D8B1EB500F26D964256943B1FBF0F1E4
:10761000A167881A1B686430584390FBF5F042F26A
:10762000107390FBF3F05843E04B984200DDE048C4
:10763000914210D0DF4900EB0012DF4B08600A21B5
:1076400092FBF1F21A6000EBC00202EB001090FB1B
:10765000F1F0DA49086030BD70B5CC4CA07994F8EF
:107660002810884211D204F1CC05284410F8011CDE
:1076700011B10020FEF7EAFEA079295C11B10120CA
:10768000FEF7E4FEA079401CA07170BD70B5BF4D3F
:10769000A879012816D905F1CC04204410F8011C62
:1076A00011B10020FEF7D2FEA879401EC0B2A87129
:1076B000204410F8011C002904D0BDE870400120CE
:1076C000FEF7C4BE70BDB148417F31B190F82210C1
:1076D000112902D1122180F82210817F002906D0C1
:1076E00090F82210122902D1132180F8221070473D
:1076F00070B5A64C05232046E17F90F8240041B1E7
:10770000224692F820506A1CD2B2814206D1E37719
:107710000BE0E377401F84F8200008E0491CE17784
:10772000854202D184F8203001E084F8202014F84A
:107730001F0FE070FFF7C7FFE17821700120FEF70F
:1077400085FE6078E070FFF7BEFFE1786170BDE80C
:1077500070400020FEF77ABE8C4901F180004A7E1D
:10776000012A01D04A6F01E002684A67CA67012115
:107770001022C0E902214160704710B5112101209B
:10778000FEF764FE8E4881490078C86302F0A2FCCF
:107790001121BDE810400020FEF758BE10B512219F
:1077A0000120FEF753FE864878490078C86302F04E
:1077B00091FC1221BDE810400020FEF747BE814831
:1077C00010B50078002807D0FFF73AFDBDE810405B
:1077D0004FF4967002F07EBC10BD70B56B4CE07A31
:1077E0000028A06B01D0401EA063012528B120799C
:1077F00070B10020207104210DE0A07B4FF0040146
:1078000020B10120FEF722FEE57070BD0020F9E7EF
:10781000257104210120FEF719FEBDE870405B4888
:10782000FC3002F0F1BD2DE9F05F584E0024DFF886
:107830009881DFF86891DFF894A1DFF894B1654F83
:107840007476012564A10120FEF7EAFC62A10920FB
:10785000FEF7E6FC707D01280ED161A1FEF7E0FC89
:1078600061A10920FEF7DCFC98F800107167717EB9
:10787000022901D188F80040707D02280FD15CA157
:107880000120FEF7CDFC5CA10920FEF7C9FCD9F868
:1078900000107167717E022901D1C9F80040707D26
:1078A00003280FD156A10120FEF7BAFC56A10920EA
:1078B000FEF7B6FCDAF800107167717E022901D17B
:1078C000CAF80040707D04280FD14DA10120FEF7B9
:1078D000A7FC4FA10920FEF7A3FCDBF8001071679D
:1078E000717E022901D1CBF80040707D05280ED1B0
:1078F0003BA10120FEF794FC47A10920FEF790FC74
:10790000474801687167717E022900D10460707D6B
:1079100006280ED143A10120FEF782FC43A10920D5
:10792000FEF77EFC434801687167717E022900D131
:107930000460707D07280ED13AA10120FEF770FC8B
:107940003DA10920FEF76CFC134801687167717E48
:10795000022900D10460707D08280ED131A10120D8
:10796000FEF75EFC36A10920FEF75AFC3648016896
:107970007167717E022900D10460707D092876D17B
:1079800032A1012066E072E0D103002060050020F2
:10799000D503002018040020E8030020DC030020A9
:1079A0000C040020B903002008040020801A0600FF
:1079B00070F30500FC030020100400201C040020CC
:1079C000C0030020C9030020D2030020E0030020F0
:1079D000E40300204D07002020202020202000006C
:1079E00020746F74616C0000637265647300000042
:1079F000202067616D65000073746172747300000C
:107A000020636F696E730000206C6566740000006F
:107A100072696768740000007265706C61730000C1
:107A2000F00300206E756D6265720000736C616D0D
:107A300073000000EC0300206562616C6C73000051
:107A400074696C7473000000F40300206176657241
:107A500061670000FEF7E4FBFEA10920FEF7E0FBF2
:107A6000FE4801687167717E022900D10460707D53
:107A7000B17D88420FD1FAA10120FEF7D1FBFAA116
:107A80000920FEF7CDFB4FF0FF307067F8484460E7
:107A9000707E012817D0AFF2C0011120FEF7C0FBA5
:107AA000716F002902DB1620FEF776FB706C401E1A
:107AB0007064FFF79CFA707E012811D0022811D063
:107AC000032811D000E07575AFF2F4010920FEF72C
:107AD000A7FBAFF2FC01BDE8F05F1920FEF7A0BBE9
:107AE0003D70AFE67576FBE7707DB17D884201D1D0
:107AF0007575A7E6401C7075A4E6DD4810B58038A2
:107B00000146447EC97C01220023012C02D019B118
:107B1000C26702E041B1C374C367C16F4167D44813
:107B2000C0E90223426010BDC274F1E7D148007879
:107B300000280AD0CE490022803900EB4000CA70EC
:107B4000886301F1FC0002F05FBC704710B5C84CBF
:107B5000803CE07800280DD104F1FC00007802F0B0
:107B6000EFFCA07B4FF0040128B10120FEF76EFC72
:107B70000120E07010BD0020F8E72DE9F041BE487B
:107B8000BB4D0078803D40B9BC48696F814204DD3F
:107B900091FBF0F200FB12106867B94C686F216826
:107BA000884225DDB74E307808B1FFF708FEB64FA2
:107BB000686F396888421CDD2160B44C21688842B6
:107BC00015DD307808B1FFF7FAFD20683860B04F56
:107BD000686F396888420CDDFFF7F1FD307818B91D
:107BE000FFF7EDFDFFF7EBFD38682060686F386048
:107BF000CAE42060C8E470B59D4C0120803C642537
:107C0000A064206D606790FBF5F105FB1100E06456
:107C1000E17B884201D1FFF713FBA06C401CA064FC
:107C2000217C88420AD8022804D0032804D0A06E00
:107C30006067E8E7A06DFBE7206EF9E770BD8C4A4E
:107C400010B5803A0023516F491E5167906CC2E90C
:107C5000123001230F280AD0082819D902240E282F
:107C60000BD0002908D100F00700546714E0002968
:107C700002D103209364506710BD39B992F83700E0
:107C8000012802D05467946410BD5367936410BDFB
:107C90000029FCD1401C5367906410BD0F2803D00D
:107CA000082803DD02207047032070470120704739
:107CB00010B578486E4C0121803C0068E0630020DC
:107CC000FEF75CFFE06B02F005FA01210020FEF7F1
:107CD00055FFE06B400002F0FDF901210020FEF7A6
:107CE0004DFFE06B400002F0F5F903210020FEF7A4
:107CF00045FFE06B02F0EEF902210020FEF73EFFA7
:107D0000DC20E063BDE8104002F0E4B95848624965
:107D10008038407C022801D8112000E00120FEF7C5
:107D20007FBA10B5524C803C607C0228AFF25831CB
:107D300014D81120FEF774FAAFF264311920FEF75F
:107D40006FFA607C022803D91620216EFEF724FA10
:107D5000607C032817D91E20A16E10E00120FEF7D9
:107D60005FFAAFF28C310920FEF75AFA0620216D36
:107D7000FEF712FA607C012805D9A16D0E20BDE83E
:107D80001040FEF709BA10BD10B544A10120FEF75E
:107D900047FA4448007808B143A100E044A1092013
:107DA000FEF73EFA324C803CE079D8B142A1112076
:107DB000FEF736FAAFF2E0311920FEF731FAE0793A
:107DC00090B1012812D03E4801681E20FEF7E4F968
:107DD000E079401CC0B20321B0FBF1F201FB1200BC
:107DE000E07110BD37A1E2E73848EDE73848EBE72E
:107DF00070B5274E1E4C214D3068803CA84228DDCE
:107E0000206FA84214D1AFF230412348FBF70EFF98
:107E100021490120FEF704FA1F490920FEF700FA64
:107E20001D491120FEF7FCF91B491920FEF7F8F94E
:107E30003068216F90FBF1F106206167FEF7ACF925
:107E40001048007820B111480168A94246DD41E0A0
:107E500069E05CE073636F72652000000C04002031
:107E6000202064617461000020646F6E6520000052
:107E7000E0050020BA030020C803002040420F00A4
:107E800000040020C503002020040020140400206A
:107E900004040020300400204B0A00202065787480
:107EA00072610000C203002067616D652020000040
:107EB00062616C6C20200000616E642061740000BF
:107EC0001C0400202020617420200000FC030020FE
:107ED00010040020206F91FBF0F161670E20FEF787
:107EE0005BF9FE480168A94203DD206F91FBF0F1C8
:107EF00061671620FEF750F9F9480168A94203DDD1
:107F0000206F91FBF0F161671E20FEF745F9206FAD
:107F1000012812D00A2190FBF1F02067BDE87040E3
:107F2000F04802F071BA0E20616FFEF735F91620A5
:107F3000616FFEF731F9616FE6E72567EEE770B52F
:107F4000E94CA07C00285DD0E84D216DA9420CDDF4
:107F5000206FA84204D1AFF280510120FEF760F9F2
:107F6000216F206D90FBF1F161670620FEF714F997
:107F7000A16DA9420CDD206FA84204D1AFF2A85137
:107F80000920FEF74DF9216FA06D90FBF1F16167BB
:107F90000E20FEF701F9216EA9420CDD206FA842E8
:107FA00004D1AFF2CC511120FEF73AF9216F206EC7
:107FB00090FBF1F161671620FEF7EEF8A16EA94281
:107FC0000CDD206FA84204D1AFF2F4511920FEF766
:107FD00027F9216FA06E90FBF1F161671E20FEF77B
:107FE000DBF8206F012809D00A2190FBF1F020670F
:107FF000BC480C30BDE8704002F006BAB9482567AD
:108000001830F7E770BD2DE9F041B74C207F00280C
:1080100074D1AFF23C61B648FBF708FE94F8370024
:108020000025B24F0126022810D0E17A002965D13F
:10803000042863D0207DA17C08435FD1E07E002826
:108040007DD0E576207A00287AD0C2E0A64880303C
:10805000006B8047207D002850D1A648007800287A
:108060004CD0A3490120FEF7DBF8A1490920FEF717
:10807000D7F89F491120FEF7D3F89D491920FEF744
:10808000CFF8062002F05CFA072002F059FA04202B
:1080900002F056FAE07EDFF86082D8B1E57603217F
:1080A0000020FEF7D3F998F8000028B1A07C18B1A1
:1080B0002767FFF744FF55E00620216DFEF76CF8B7
:1080C0000E20A16DFEF768F81620216EFEF764F809
:1080D000A16E44E08948E676007880B1E674E07DE0
:1080E000401CC0B2E07502280AD9E571FFF74CFECA
:1080F0007C480C3802F088F9E57533E070E0E574EF
:1081000003210120FEF7A2F998F800007C4D30B160
:108110002868B84203DD2767FFF76AFE22E00620E1
:108120002968FEF739F87748007878B17648016811
:108130000E20FEF731F869480168162001E02DE0B5
:1081400014E0FEF729F86648016808E00E20296867
:10815000FEF722F816202968FEF71EF829681E206F
:10816000FEF71AF85F4826753C3035E0607C012840
:1081700006D0022807D0032808D0042809D028E018
:108180005B49012007E05A49092004E058491120C1
:1081900001E057491920FEF743F81AE02767207AD3
:1081A000B0B9607C012806D0022807D0032808D087
:1081B000042809D00CE00620216D07E00E20A16DF7
:1081C00004E01620216E01E01E20A16EFDF7E4FF01
:1081D000E676444826754830BDE8F04102F014B90F
:1081E00006E5414901F180004A7E012A01D04A6F2B
:1081F00001E002684A67CA674449C1604449816036
:1082000042F21071416070472DE9F05F364E002553
:1082100001277576DFF8F090DFF8C0A0DFF8E08086
:10822000DFF8BCB086F8257006F18004AFF658017F
:108230000920FDF7F5FF96F82500012811D1AFF6CA
:108240001C01FDF7EDFF33A10920FDF7E9FF334BDA
:1082500018787067FFF780FA96F874001870082095
:10826000A06096F8250002280ED12DA10120FDF76F
:10827000D7FF2DA10920FDF7D3FF2D4B186870679C
:10828000FFF7AFFF706F186096F8250003280ED136
:1082900028A10120FDF7C4FF23A10920FDF7C0FF9D
:1082A000264B18687067FFF79CFF706F186096F890
:1082B000250004280ED122A10120FDF7B1FF1AA14B
:1082C0000920FDF7ADFF204B18687067FFF789FFA5
:1082D000706F186096F82500052837E0200400200C
:1082E00000040020740600206005002040420F00BA
:1082F0004B0A0020C6030020C8030020B903002059
:1083000004040020C503002014040020803801006C
:10831000301B0F0062616C6C73000000BB03002017
:108320002066697273740000746872657368000077
:10833000FC0300207365636F6E640000100400206E
:1083400020746869726400001C04002010D1F8A138
:108350000120FDF765FFAFF204510920FDF760FF32
:10836000D8F8000043467067FFF73BFF706F186056
:1083700096F82500062812D1EFA10120FDF750FF45
:10838000EFA10920FDF74CFFEF4B18787067FFF75E
:10839000E3F996F8740018701E20C4E9020596F8F7
:1083A0002500072812D1E9A10120FDF739FFE9A135
:1083B0000920FDF735FFE94B18787067FFF7CCF916
:1083C00096F8740018702820C4E9020596F8250074
:1083D000082811D1E2A10120FDF722FFE2A1092026
:1083E000FDF71EFFDFF888C39CF80000F074FFF76C
:1083F00084FBF07C8CF8000096F82500092811D148
:10840000DCA10120FDF70CFFDCA10920FDF708FF2E
:10841000DFF870C39CF80000F074FFF76EFBF07C8F
:108420008CF8000096F825000A2828D1CCA101205C
:10843000FDF7F6FED4A10920FDF7F2FEDFF850C3E8
:108440009CF80000F074FFF758FB9CF8000001282E
:1084500012D1F07C80B9CF4AD8F8001091420BDDE0
:10846000CD49C8F80010CD49C9F80010CC49CAF868
:108470000010CC49CBF80010F07C8CF8000096F886
:1084800025000B2813D1AFF6A8210120FDF7C8FE67
:10849000C5A10920FDF7C4FEC54B18787067FFF72A
:1084A0005BF996F8740018700520C4E9020596F887
:1084B00025000C2811D1BFA10120FDF7B1FEBFA1FD
:1084C0000920FDF7ADFEDFF8FCC29CF80000F07457
:1084D000FFF713FBF07C8CF8000096F825000D28C0
:1084E00011D1B9A10120FDF79BFEB9A10920FDF72B
:1084F00097FEDFF8E4C29CF80000F074FFF7FDFA85
:10850000F07C8CF8000096F825000E2811D1B3A15C
:108510000120FDF785FEB3A10920FDF781FEDFF8FC
:10852000CCC29CF80000F074FFF7E7FAF07C8CF8FE
:10853000000096F825000F2811D1ADA10120FDF70C
:108540006FFEADA10920FDF76BFEDFF8B4C29CF809
:108550000000F074FFF7D1FAF07C8CF8000096F878
:10856000250096F82710884205D396F826108842F1
:1085700001D2606B804796F8250096F82610884255
:108580000ED1A0A10120FDF74BFEA0A10920FDF70F
:1085900047FE4FF0FF3070676560707E012818D08D
:1085A000AFF6CC311120FDF73BFE716F002902DBE5
:1085B0001620FDF7F1FD706C401E70640BD0FEF7C5
:1085C00016FD707E012811D0022844D0032846D021
:1085D00001E086F825708BA10120FDF721FEAFF6A2
:1085E0000841BDE8F05F0920FDF71ABED4E901108B
:1085F000421AF06F824201DAE06800E0084420602D
:1086000096F82500052823D1206890FBF1F0484317
:1086100044F62061C8F80000884203DD421AC9F818
:10862000002001E0C9F8005047F23051884203DDD4
:10863000411ACAF8001001E0CAF8005049F640415A
:10864000884203DD401ACBF8000001E0CBF800506F
:1086500070480770EAE5E06820607776F8E796F8FA
:10866000250096F82610884202D186F82570DDE5AF
:10867000401C86F82500D9E510B56748674C0321F2
:108680000068E0630020FEF779FAE06B01F022FD5C
:1086900002210020FEF772FAE06B01F01BFD0121C0
:1086A0000020FEF76BFAE06B01F014FD02210020C0
:1086B000FEF764FAE06B01F00DFDE06B01F00AFDDE
:1086C00001210020FEF75AFAE06B01F003FD0321BF
:1086D0000020FEF753FABDE81040012001F030BF42
:1086E0004F4B5048002119800268002A15D04B4892
:1086F000406F904211DD4C4A491C19801268002AD3
:108700000BD0904209DD494A491C19801268002AA1
:1087100003D0904201DD491C198070473F49886CA5
:108720000F2803D0082802D9022084E080E081E0ED
:10873000202068696768000020206175746F000060
:1087400070657263656E0000B903002020206261CD
:108750006C6C00007361766520200000BA03002075
:10876000656E61626C65000034204853544400001B
:10877000C5030020202073686F770000687374645D
:1087800020200000C60300206D696C696F6E000038
:10879000C803002040420F00E0E60B0020120A0050
:1087A000603D0800A068060074696C7473200000C6
:1087B000D30300202069646C65200000616E696D40
:1087C00061740000CA0300202066617374200000F9
:1087D000626F6E7573200000C303002020736B6905
:1087E0006C6C000073686F7420200000CE030020C2
:1087F0005475726E6D7400004D6F6465202000002A
:10880000D50300202073657475700000646F6E6579
:10881000202000004D0700203004002060050020CB
:10882000B4030020FC030020100400201C040020DE
:10883000032000E00120886470477047F74810B5B6
:108840000168F84C491C0160F5480078A06494F870
:108850002A006067FFF7F3F994F8740084F82A009F
:10886000F148007808B1FFF723FAA06C002805D082
:10887000FEF7CDFCA06C401EA064F7E710BD2DE90B
:10888000F047E84E0025DFF8A493DFF8A4A375763F
:108890004FF00F0806F180040127AFF6C4610920EC
:1088A000FDF7BEFC96F82D00012814D1E1A1FDF7DB
:1088B000B7FCE2A10920FDF7B3FCD94B187870672B
:1088C000FEF74AFF96F874001870FFF7E7F986F88C
:1088D0002A00C4E9028596F82D00022815D1D9A1F5
:1088E0000120FDF79DFCD5A10920FDF799FCD74B90
:1088F00018787067FEF730FF96F874001870FFF76D
:10890000CDF986F82B00C4E9028596F82D000328DE
:1089100011D1CFA10120FDF783FCCFA10920FDF7E4
:108920007FFCDFF83CC39CF80000F074FFF7E5F82B
:10893000F07C8CF8000096F82D00042811D1C9A114
:108940000120FDF76DFCC9A10920FDF769FCC94BA9
:1089500018787067FEF700FF96F874001870C4E985
:10896000028596F82D00052811D1C3A10120FDF73D
:1089700057FCC3A10920FDF753FCDFF8ACC29CF8FB
:108980000000F074FFF7B9F8F07C8CF8000096F85E
:108990002D00062813D1AFF224210120FDF740FC61
:1089A000AFF6BC710920FDF73BFCDFF8DCC29CF898
:1089B0000000F074FFF7A1F8F07C8CF8000096F846
:1089C0002D00072811D1B1A10120FDF729FCA5A197
:1089D0000920FDF725FCDFF8BCC29CF80000F0740C
:1089E000FFF78BF8F07C8CF8000096F82D00082833
:1089F00011D1A6A10120FDF713FCA7A10920FDF7C5
:108A00000FFCDFF89CC29CF80000F074FFF775F8CB
:108A1000F07C8CF8000096F82D00092818D19BA155
:108A20000120FDF7FDFB9FA10920FDF7F9FB707EFA
:108A3000012802D12168C9F80010D9F80000706738
:108A4000F0674FF47A704EF66021C4E9021060605E
:108A500096F82D000A2811D194A10120FDF7E0FB22
:108A600087A10920FDF7DCFBDFF848C29CF8000075
:108A7000F074FFF742F8F07C8CF8000096F82D00B7
:108A80000B2812D1AFF228310120FDF7C9FB72A1EA
:108A90000920FDF7C5FBDFF820C29CF80000F07448
:108AA000FFF72BF8F07C8CF8000096F82D000C28CE
:108AB00011D182A10120FDF7B3FB6CA10920FDF7C4
:108AC000AFFB804B18787067FEF746FE96F874008F
:108AD00018700820A06096F82D000D2811D17AA1F9
:108AE0000120FDF79DFB7AA10920FDF799FBDFF836
:108AF000E8C19CF80000F074FEF7FFFFF07C8CF8F2
:108B0000000096F82D000E2812D1AFF2AC310120F2
:108B1000FDF786FB71A10920FDF782FBDFF8C4C1D8
:108B20009CF80000F074FEF7E8FFF07C8CF8000081
:108B300096F82D0096F82E1088420FD16AA10120D8
:108B4000FDF76EFBAFF23C310920FDF769FB4FF0FA
:108B5000FF3070676560707E012817D0644911206E
:108B6000FDF75EFB716F002902DB1620FDF714FB99
:108B7000706C401E70640BD0FEF739FA707E0128CD
:108B800010D002281BD003281DD001E086F82D70DC
:108B900055A10120FDF744FBBDE8F04754490920E9
:108BA000FDF73EBBD4E901010A1AF16F8A4201DAEE
:108BB000E06800E0084420608AF800706DE6E06834
:108BC00020607776F8E796F82D0096F82E10884208
:108BD00002D186F82D7060E6401C86F82D005CE618
:108BE0001048F03001F010BC10B50E4C0020404988
:108BF00020720120FDF714FB3D490920FDF710FB11
:108C00000620216DFDF7C8FA207C012805D9A16D49
:108C1000BDE810400E20FDF7BFBA10BDE0030020F4
:108C2000BD03002060050020CC03002018040020B4
:108C30004D07002020206C6566740000636F696E2C
:108C4000730000002072696768740000BE03002092
:108C500020636875746500006D61746368000000CE
:108C6000BC03002063726564697400006C696D69FF
:108C700074000000D00300202020636F696E0000A4
:108C8000736F756E64730000C703002073706563B3
:108C9000696C0000C20300206F7665727264000088
:108CA000C103002061776172640000002073636F6C
:108CB00072650000CD030020C40300206578626166
:108CC0006C6C0000D1030020202048535444000065
:108CD0006177617264200000C90300206164766ED0
:108CE00063650000D40300206F7074696F6E00002C
:108CF000D87900082DE9F041FE4D95F8370002289B
:108D00007ED0E87A00287CD0E878A97A084379D028
:108D1000287A38B1082001F013FC092001F010FC7A
:108D2000FFF762FFF34CA87A00260127803478B160
:108D3000AE7202210020FDF789FB85F83770E069EB
:108D40008047E87C40B14FF4FA6001F0C3F903E0DA
:108D5000A06A8047E06A8047E748007801F0F0FBAE
:108D6000EE72A87B002862D1687C297C88425CD1A5
:108D7000E249287B0978884207D2401CC1B2297396
:108D80000820FDF709FA6F7451E001210020FDF77A
:108D90005DFB022085F83700D9480078A0B10A2091
:108DA000A864FAF7FEFA95F848104843C1B2E9738F
:108DB0000820FDF7F1F9E87B18B900210720FDF73D
:108DC000EBF9FEF718FF04E0AFF274610720FDF73E
:108DD00027FA286D20616867287C01281ED0FEF7DD
:108DE000CCFE2169A86D014421616867287C0228B6
:108DF00014D0FEF7C2FE2169286E0144216102E011
:108E00003FE031E02AE06867287C032806D0FEF7BF
:108E1000B4FE2169A86E014421616867FEF7ADFECA
:108E2000FEF7CFFBF9F7BBFF01E0401C687495F833
:108E30003700022825D0A0698047FDF795FBA87B65
:108E400038B104210120FDF701FBA87B401EA87367
:108E500001E0FEF76BFE206A804701E0FEF776FE38
:108E600095F8370002280CD04FF42F70E86301F01A
:108E700031F905210020FDF781FEBDE8F041FDF745
:108E8000EEBFA0480078002805D0BDE8F0419A4820
:108E9000843801F0B9BABDE8F081704770B50E466C
:108EA0000546012415E0295D032905D99648007877
:108EB000001F052802D20221002000E00220FDF759
:108EC0005DFE9249305D0968484301F003F9641C76
:108ED000E4B22878A042E6D270BD8B4810B5007885
:108EE000092813D903210020FDF748FEFA2001F0DC
:108EF000F1F802210020FDF741FEFA2001F0EAF826
:108F00000121BDE810400020FDF738BE7A49BDE8D8
:108F100010401C31A1F11000C0E710B50121002064
:108F2000FDF794FA7A480078FEF7B8FE714C04F821
:108F30002A0F78480078FEF7B1FE60706D488030E7
:108F4000C06980470020A0722A3CFFF7C6FFFDF7EA
:108F500018F900210620FDF71FF96948007850B183
:108F60000A20A064FAF71DFAA16C48430146A064E8
:108F70000820FDF711F96848007820B167480178AA
:108F80001020FDF709F9607F28B194F8210080F0E6
:108F9000100084F82100A07F20B114F8210F80F088
:108FA0002000207057480078002805D05248BDE8BE
:108FB0001040843801F028BA2FE6704710B5574C9E
:108FC000207800280FD0401E2070534800780028D9
:108FD00009D0FF211020FDF7BDF82178BDE8104031
:108FE0001020FDF7D9B818E670B5424C4C48002661
:108FF000A664007818B149480078002878D994F818
:109000003700022803D0607C012856D098E03A4807
:109010002438007801F094FA37486C38007801F071
:109020008FFA35486038007801F08AFA32485438AF
:10903000007801F085FA30484838007801F080FA6D
:10904000FDF79FF82B4D803568698047A8698047F8
:10905000082084F837000121FDF79EF8FFF7AEFFE6
:10906000267503210020FDF7F1F904210020FDF70A
:10907000EDF901210846FDF7E9F902210020FDF78D
:10908000E5F9FFF7F9FA686A8047FDF76DFA286A93
:1090900080474FF42F70E06301F01CF80521002099
:1090A000FDF76CFDFDF7DBFE1E4800686065E065BE
:1090B0006066E066FEF73AFD0BE0207C04283FD2B4
:1090C000207B01283CD110480078102838D0FFF7C9
:1090D00075FF207C1449401CC0B220740A68521CE1
:1090E0000A60012834D0FFF7C7FA207C02281DE06F
:1090F00036E0000060050020D4060020BB030020FD
:10910000C4030020CA0300202404002030040020EF
:10911000BD030020BE030020C7030020D2030020AF
:10912000D0030020FC030020DC03002013D0032820
:109130004FF0000112D01E20BDE87040FDF72CB8A2
:10914000012084F83100BDE87040F74801F05CB9B7
:1091500000210620F0E700210E20EDE71620EBE7C6
:1091600070BD10B5F14C224694F8353092F8362097
:10917000012B0ED0805C84F82200C1B294F8330039
:10918000FDF764F994F8330028B1002084F8330027
:1091900043E5885CEFE70120F8E770B500240D4651
:1091A000224608E0295D04F10104E4B20029F9D166
:1091B00002F10102D2B28242F4D304E0641CE4B2B0
:1091C0000620FDF743F9295D0029F7D170BD2DE98F
:1091D000FF5F0124D54F1E469046FC748146A3468E
:1091E000254602EB060A7867444504D8601EC0B2E3
:1091F0000199FFF7D2FF282000F06CFFB9F1000FB2
:1092000002D0786FFEF70DF9282000F063FFB4421A
:1092100005D9A01B401EC0B20199FFF7BEFFA245B1
:1092200002D10020F87408E0012C03D0F87C20B1B2
:10923000641C03E087F813B0FAE7641E6D1CEDB2FE
:10924000E4B2142DD0D9BDE8FF9F2DE9F047B74C0B
:1092500001251E4617468846814684F83550FDF79D
:10926000B1F9B3A1B648FAF7E1FCFEF74FFD4FF4B0
:109270007A7000F02FFFFDF777F9A5640121002037
:10928000FDF77CFC02210120FDF7E0F83C2000F016
:1092900021FF01210020FDF771FCFDF765F9022196
:1092A0000020FDF7D3F83C2000F014FFA06C401C18
:1092B000A0640828E2D933463A4641464846FFF7BB
:1092C00086FFFEF72EFD84F83650002084F8330028
:1092D00095480C3001F098F8BDE8F047FDF77DB9EE
:1092E00070B5924C94F8310001282BD1207A28B126
:1092F000082001F025F9092001F022F9A07A0025C3
:1093000020B1A57202210020FDF7A0F80E2001F087
:1093100017F9022001F014F984488030C0698047B1
:10932000E07C18B14FF4FA6000F0D4FE0B2001F09D
:1093300007F9E572A573022084F83700FFF754FEA1
:1093400084F8315070BD7F4810B50168774C491CD6
:1093500001607D48007860B17C480078A06494F892
:109360002A006067FEF76BFC94F8740084F82A000A
:109370000BE077480078A06494F82B006067FEF754
:109380005EFC94F8740084F82B00A06C28B1FDF703
:109390003EFFA06C401EA064F8E76E4800780028ED
:1093A00003D0BDE81040FEF783BC36E42DE9F04160
:1093B000694801786948006831B169490978092923
:1093C00002D3C0F3470600E0C6B2584D65494FF4DA
:1093D0007A77687BE0B36C7988461DE06C710CE0AD
:1093E000FDF7B7FE3846FEF71CF8304600F072FE77
:1093F000FDF7D4FE6879401E687168790028EFD1C6
:10940000D8F8000000F066FEA879012802D9FEF71E
:109410003DF901E0401EA871A8790028DED13AE5A7
:10942000AC79FDF796FE07E03846FDF7FAFF3046C7
:1094300000F050FE641EE4B2002CF5D1FDF7AEFE44
:109440006879401E6871D8F8000000F043FE01E022
:10945000FFE7884668790028E2D11CE5704770B5BF
:10946000324C002604F1D70184F83360881FFFF7DF
:1094700015FD3D4D2878E0742E7042F21070606743
:10948000FDF7CFFFE07C2870BDE87040C82000F0F9
:1094900021BE10B502210020FCF7D8FF3348007828
:1094A000002805D02048BDE81040783800F0ACBF57
:1094B00082E52F4810B501681C4C491C0160022050
:1094C00084F8370001210020FCF7C0FF02210120B1
:1094D000FCF7BCFF04F5BA70007801F031F8FEF734
:1094E00035FBF9F75CFC1E4800780A2815D21D48A8
:1094F00003210068E0630020FDF740FBE06B4000C3
:1095000000F0E8FD02210020FDF738FBE06B00F0E1
:10951000E1FD01210020FDF731FB42F2107000F067
:10952000D9FDBDE81040B4E7C80600206005002062
:10953000796F7520646177697A6172640000000058
:109540004B0A0020E4030020BC030020BD030020E0
:10955000BE030020CC030020C30300202804002009
:109560002404002030040020CD030020CA03002082
:10957000EC03002070B5DA4CA07A00283CD194F8B6
:109580003700022838D0D7480078B0B3617A012577
:10959000491CC9B26172884239D1FEF7D7FA00205E
:1095A0006072D1480168491C0160A5720221012046
:1095B000FCF74CFFFA20E06303210020FDF7DEFA00
:1095C000E06B00F087FD03210020FDF7D7FAE06B88
:1095D00000F080FD03210020FDF7D0FAE06B00F0E1
:1095E00079FD01210020FDF7C9FA04F18000C06B6C
:1095F0008047042084F8370070BDFFE7022084F81C
:109600003700BDE8704001210020FCF71FBFB748BC
:109610002572007800F094FFB4480C30007800F018
:109620008FFFB24800F0F0FEB0480C3000F0ECFEC6
:10963000AFA10120FCF7F4FDBDE87040AEA1092008
:10964000FCF7EEBDA649487A002801D0401E4872BA
:109650007047A349002008757047A14890F8301062
:1096600019B1002180F830107047012180F83010C6
:109670009B488030006C0047994A10B5002302F1E6
:109680008001102830D2DFE800F02F080B0E1131D6
:109690001414171A1D1D1F22292CFEF729F825E086
:1096A000FEF79BF822E0FEF76FFB1FE0FEF7A0FB42
:1096B0001CE0FEF744FC19E0FFF7C4FF16E0FFF7DB
:1096C00093FA13E0137511E0FFF7C7FF0EE00320D4
:1096D000FDF794FB50B1FFF703FE07E0486C8047AD
:1096E00004E0FFF7D6FE01E0896C8847002063E4C0
:1096F000032811D005DC58B101280BD002280FD166
:1097000021E6042809D0052808D00F2808D1D0E682
:1097100000F010BCFFF792B866E42BE7FFF7EABA57
:10972000704770B576480024784904707548012563
:1097300004707548047005200870754879A105709B
:109740007448046074480460744805707448057077
:109750007B48FAF76BFA7B487E49032204707A480B
:10976000994B0470794805707948057040F6C4102B
:10977000086079487B49047078480470784808602C
:109780007A49794808607A487B49046079480860DA
:109790007A487C4905707A4805700F2008707A482D
:1097A00085490570794804707948027079480470D9
:1097B0007948046079480460794804607948046015
:1097C0004948046078480570784804607848057016
:1097D000784808607A49794808607A490C70C8214D
:1097E00019707A4B1C707A4B1D707A4D44F62063C9
:1097F0002B60794B794D1C704FF47A732B60784B4A
:109800001860794B77481860364802707748784A74
:1098100004704B201060774A1060774A10607748D8
:109820000160E9E62DE9F0412D4C0126002504F800
:10983000136F73A1C4F83550C4F83950C4F861509F
:10984000C4F865507048641CFAF7F0F904F8095C34
:1098500025704FF00F0804F8148C66700A20A07071
:1098600004F8075C1E4FA566E570803725713D60E2
:109870006571A571022084F82300E671257260A14C
:1098800007F15D007D60FAF7D1F9A5626572A572F6
:10989000E5722573FF206073A57384F80F80242080
:1098A000BD602074667484F813801020A074FD607D
:1098B0006575A675E67584F81880667684F81A8052
:1098C00052A107F16500FAF7B1F93D615148E5761B
:1098D00065770580A5774FF416702063E5779EE5E0
:1098E00060050020D3030020F40300209806002028
:1098F0002077686F61680000627562626120000015
:10990000B8030020B9030020BA030020BB030020E5
:10991000BC030020E0030020E4030020BD0300207E
:10992000BE03002053797374656D31204350552078
:109930002041524D20206D6F64656C2000000000B6
:10994000DB090020BF030020C5030020C603002060
:10995000C7030020D8030020C8030020D403002040
:10996000C0D40100FC03002070820300000400202A
:10997000DC03002000E2040004040020C9030020EE
:10998000CA030020CF030020C4030020D00300201E
:10999000D1030020D2030020E8030020EC030020C4
:1099A000F003002008040020CC0300200C04002059
:1099B000CD03002020BF020010040020C045040099
:1099C00014040020CE030020C0030020C1030020A7
:1099D000C203002018040020C3030020F803002065
:1099E0001C04002090D0030020040020D503002098
:1099F0002C0400203004002028040020340400201F
:109A00006E756C6C000000004B0A0020322E34335F
:109A100000000000B403002010B5FDF74DFA032844
:109A200006D028B1FDF736FAFD490020087010BDB8
:109A3000012010BD2DE9F041FA4FFB4D4FF496780F
:109A4000C7F800802878F94E0124002868D0C0EBC0
:109A5000C00081190920C91FFCF7E2FB23E0FDF7D4
:109A60006BFA012804D002284AD003281BD14BE00E
:109A7000EB49002008702878062814D2DFE800F0AF
:109A800040030B0E111B24B100242046FCF70CFCF4
:109A900009E00124F9E7FCF7B0FD04E0FDF7BEF8AA
:109AA00001E0FDF7BDFA3868401E3860401CD6D191
:109AB0000120BDE8F081FFF734FEDD48DD4A006893
:109AC000A0F59C4120391160DB4AA0F5EA4130390C
:109AD0001160DA49A0F51C40403808600120687028
:109AE00003210020FDF74AF8D5490920FCF798FB2F
:109AF0004FF4FA7000F0EEFACC491C310920ABE7C4
:109B0000FCF73FFB0020D4E7C7F800802878012449
:109B10000621401CB0FBF1F201FB1200287094E713
:109B2000C749092098E72DE9F041BE4F4FF49670E0
:109B3000C4A138600920FCF773FBC44CDFF8E8824D
:109B4000207808F1020800EB800101EBC0014144DC
:109B50001120FCF765FB267800252FE0FDF7ECF9D6
:109B6000012804D0022815D0032827D115E0B848D1
:109B7000112105702078401CB0FBF1F201FB1200AE
:109B800000EB800101EBC001207041441120FCF783
:109B900047FB13E0257000208BE7AEA10920FCF7FE
:109BA0003FFBACA11920FCF73BFB2078B04204D06E
:109BB000F9F74BF89C49012048703D603868401E19
:109BC0003860401CCAD1012073E72DE9F05FA3493A
:109BD00001240020DFF88892A24DDFF88C82A34E8A
:109BE000A34F08704FF0050A9AA10920FCF718FB53
:109BF000012C10D0022C19D0032C2ED0042C40D0D4
:109C0000052C5AD0062C76D0072C71D0082C70D099
:109C1000092C6FD0D4E097A10120FCF701FB97A19C
:109C20000920FCF7FDFADFF85CB209E096A10120FB
:109C3000FCF7F6FA91A10920FCF7F2FADFF850B22E
:109C4000DBF800002860D9F800008047296832203E
:109C5000CBF800103860C8202AE08EA10120FCF764
:109C6000DFFA8EA10920FCF7DBFADFF838B29BF8A7
:109C700000002860D9F80000804728788BF80000A1
:109C800012E084A10120FCF7CBFA7CA10920FCF7AB
:109C9000C7FADFF814B2DBF800002860D9F800003A
:109CA00080472968CBF80010642038604FF4967024
:109CB000C8F80000C6F800A082E07CA10120FCF7F3
:109CC000AFFA7CA10920FCF7ABFADFF8F0B19BF802
:109CD00000002860D9F80000804728788BF8000041
:109CE0000A2038603220C8F80000012038E002E085
:109CF0001DE037E053E072A10120FCF791FA72A158
:109D00000920FCF78DFADFF8C8B1DBF80000286005
:109D1000D9F8000080472968CBF800104FF42F7065
:109D2000386040F2DC516420C8F8001018E064A1EB
:109D30000120FCF775FA67A10920FCF771FADFF83A
:109D40009CB19BF800002860D9F800008047287873
:109D50008BF800001E20962138600A20C8F80010F9
:109D600030602DE05EA10120FCF75AFA5EA10920C7
:109D7000FCF756FA37A11120FCF752FADFF870B160
:109D800006E001210020FCF7F9FE3C2000F0A2F9DA
:109D90005848DBF8001000688142F2D010E056A16C
:109DA0000120FCF73DFA56A10920FCF739FA4FF0E3
:109DB000FF3028600020306028480078012818D043
:109DC00024A11120FCF72CFA2968002902DB1620B7
:109DD000FCF7E2F913490868401E086009D0FDF756
:109DE00006F91E49087801280DD0022815D003284D
:109DF00014D041A10120FCF713FABDE8F05F15A1D2
:109E00000920FCF70DBAD8F8001030680A1A3E494C
:109E100009688A427ADA396879E07CE083E075E0A3
:109E200044080020480800204C070020A902002018
:109E3000040400201404002020040020000400205A
:109E40007802002073656C656374000024040020B0
:109E5000B8030020202020202020000079050020C9
:109E600070040020D4050020E8050020E40500204F
:109E7000EC0500202073636F726500006C61672041
:109E8000746D00003004002020626F6E7573000056
:109E9000280400202020636F696C0000686C642037
:109EA000746D0000C00300203404002020206C6189
:109EB0006D700000656E6120746D0000CF0300209E
:109EC000737769746368000073747220746D0000A6
:109ED000F803002064757020746D00000C070020EA
:109EE000202054696D65000063616C696272000036
:109EF0004C050020500500206578706572740000E4
:109F0000646F6E6520200000DC0500200144584885
:109F10000160012004E056483A68026001200870A0
:109F20005449487060E6092C02D0641CE4B25BE638
:109F3000012459E62DE9F047FCF723F9DFF83491C5
:109F400001214D4E89F800100D464FF0000A4FF4E4
:109F5000167889F801A04446F11D44E0FCF7ECFFB7
:109F6000012804D002282DD003283FD12CE0C5EBD6
:109F7000C50081190F460120FCF752F9072D16D2B2
:109F8000DFE805F02004070A0D101300FEF73CF986
:109F90000DE0FDF748FC0AE0FFF74CFD07E0FEF797
:109FA0006EFC04E0FFF7BFFD01E0FFF70EFE002CA2
:109FB00008DD444639460120FCF732F9AFF26C1156
:109FC000112011E0002411E02C486D1C444600785B
:109FD000EDB208B1072000E00620A84200D100251C
:109FE000C5EBC50081190120FCF71AF9201EA4F168
:109FF0000104B3DC99F801004C4658B120A10120BE
:10A00000FCF70EF920A10920FCF70AF9F8F7C7FEC2
:10A0100084F801A04FF4487000F05CF81C4902205D
:10A020000870FCF7AEF81B48007828B11A48017890
:10A030001020FCF7B1F804E0AFF2E4110F20FCF7B8
:10A04000EFF816480178BDE8F0470820FCF7A4B8FF
:10A05000134810B50168491C016001210020FCF77C
:10A06000F5F9F8F79CFEBDE81040F6F770BB00006C
:10A07000E00500204C07002078020020D4030020D7
:10A08000736176696E6700006E7672616D20000004
:10A0900097050020C7030020D2030020C40300203E
:10A0A000EC03002010B502460020F74C207001217F
:10A0B0000CE0012305E0F448007808B1084610BD23
:10A0C0005B1C40F6A6608342F5D9491C9142F0D949
:10A0D0000020F4E710B501210CE0012205E0EA4C74
:10A0E00024780CB140F6A663521C40F6A664A24246
:10A0F000F5D9491C8142F0D910BD0020E349088000
:10A10000E3490870E3490870E349087040F26D10B4
:10A11000E24908800420E24908707047E04800786E
:10A12000E04908700520DE4908707047DD48007876
:10A13000DB49087070474188D44A11808179D44A3C
:10A1400011704179D34A11700179D34A1170018895
:10A15000D24A1180D44AC16811600321D04A1170DB
:10A160007047D2480088D2490880D24800780871E8
:10A17000D14800784871D14800788871D04800886B
:10A180004880704700B50346FFF7EBFFC84840889A
:10A190001844801F82B24FF47A7092FBF0F100FBFA
:10A1A0001120C34948804FF47A7092FBF0F082B2DC
:10A1B000002A34DD08468079104482B23C2092FBAC
:10A1C000F0F100FB1120BA4988713C2092FBF0F0BD
:10A1D00082B2002A23DD08464079104482B23C2036
:10A1E00092FBF0F100FB1120B14948713C2092FB39
:10A1F000F0F082B2002A12DD08460079104482B2E3
:10A20000182092FBF0F100FB1120A94908711820D9
:10A2100092FBF0F082B2084600881044088000BD2E
:10A220009E480088A24908809B4800780871994898
:10A230000078487196480078887194480088488072
:10A240007047002008E0002100EB40029D4B03EB2B
:10A25000C2021172411CC8B22028F4DB00219A4AC4
:10A2600011607047024602B111B96FF002007047E9
:10A2700010880B88984201DD0120F8E710880B88D0
:10A28000984202DA4FF0FF30F1E710790B799842EB
:10A2900001DD0120EBE710790B79984202DA4FF0EB
:10A2A000FF30E4E750794B79984201DD0120DEE789
:10A2B00050794B79984202DA4FF0FF30D7E7907926
:10A2C0008B79984201DD0120D1E790798B79984212
:10A2D00002DA4FF0FF30CAE750884B88984201DD20
:10A2E0000120C4E750884B88984202DA4FF0FF30D3
:10A2F000BDE70020BBE730B5024610880D88431B40
:10A300001BB1002B00DA22E040E010790D79441BEC
:10A310001CB1002C00DA21E03FE050794D79431B5D
:10A320001BB1002B00DA20E03EE090798D79441BD0
:10A330001CB1002C00DA1FE03DE050884D88431B23
:10A34000002B02DA584200B230BD18B2FCE708799F
:10A350001579401B182505FB030400BF4879557982
:10A36000401B3C2505FB040300BF88799579401B01
:10A370003C2505FB030400BF48885588401B4FF46B
:10A380007A7505FB0403584200B2DDE710790D79B8
:10A39000401B182505FB030400BF50794D79401B75
:10A3A0003C2505FB040300BF90798D79401B3C25BB
:10A3B00005FB030400BF50884D88401B4FF47A759D
:10A3C00005FB040318B2BFE770B504463E480568B4
:10A3D00001E02E466D6929462046FFF743FF00281D
:10A3E000F7DC39480068854202D03748006840B938
:10A3F000354800686061344804600068FFF79BFEE0
:10A4000001E07461656170BD70B50446A088642880
:10A4100002DA6FF0010070BD002601E0701CC6B2C8
:10A42000202E07DA06EB4600264901EBC000007A31
:10A430000028F3D1202E02D14FF0FF30EBE706EBDE
:10A440004600204901EBC005A088FFF79BFE184895
:10A45000016829608188A9808079A871A0882882F4
:10A4600060786872A078E87120782872A068E86047
:10A470002846FFF7A9FF0020CDE710B51248006875
:10A4800008B900244CE021E04408002032080020F4
:10A490003B0800203D0800203F080020380800202D
:10A4A000B20300205408002058080020360800207D
:10A4B000DC0D00203E0800203C0800203A08002067
:10A4C00030080020DC0A00204C08002034480468D2
:10A4D00034480078022803D1607AFFF7CDF801E014
:10A4E000E06880472E48006840692D490860E0799F
:10A4F000012802D10020207212E0E079002802DD5C
:10A50000E079401EE071208AFFF73CFE2648016892
:10A5100021608188A1808079A0712046FFF754FFD7
:10A520001F48006818B904201E49087007E01C483D
:10A530000068A04203D01A480068FFF7FCFD10BD78
:10A5400030B505461648006810B94FF0FF3030BDF1
:10A550001348036801E01C465B6913B1187AA842EE
:10A56000F9D113B94FF0FF30F1E70D480068984278
:10A5700006D106200B49087009495869086001E0B6
:10A5800058696061002018720548006820B10448CD
:10A590000068FFF7D0FD01E0FFF7AFFD0020D6E730
:10A5A0004C080020B2030020DC0D00200100000058
:08A5B000960000008D66000812
